:10000000850186010313831606309F0003308500A7
:10001000860185308100031383128101F5010130CF
:10002000F0000530F300F2017308F1007411741050
:100030009C300102031C43288101F1080319F203DB
:10004000F10B2D28F208031D2D28700DF00DF41C66
:100050002A28F00AF2017308F100051C35287419EA
:100060003328F50A3428F5013A28741D3928F50A91
:100070003A28F5010A307502031C4328741D4228F2
:10008000741143287415851C4A28F4184A28F4145E
:100090000130F00085185128F41C5128F41001306B
:1000A000F00074185F28741D5E2874140530F3077F
:1000B0007308323C03185E280530F3006228741977
:0A00C00062287410700886001828EA
:02400E00393D3A
:00000001FF
